S01B00006F70656E62746C5F656B5F6C6D3373363936352E737265632E
S113000050110020314D0000095B0000095B000025
S1130010095B0000095B0000095B0000095B00004C
S1130020095B0000095B0000095B0000095B00003C
S1130030095B0000095B0000095B0000095B00002C
S1130040095B0000095B0000095B0000095B00001C
S1130050095B0000095B0000095B0000095B00000C
S1130060095B0000095B0000095B0000095B0000FC
S1130070095B0000095B0000095B0000095B0000EC
S1130080095B0000095B0000095B0000095B0000DC
S1130090095B0000095B0000095B0000095B0000CC
S11300A0095B0000095B0000095B0000095B0000BC
S11300B0095B0000095B0000095B0000095B0000AC
S11300C0095B0000095B0000095B0000095B00009C
S11300D0095B0000095B0000095B0000095B00008C
S11300E0095B0000095B0000095B0000095B00007C
S11300F0044B9D46C046C046C046C04603F00DFFB3
S113010004F0EEFE5011002003E00B780370491C4C
S1130110401C13005A1E002BF7D1704701E00170F8
S1130120401C13005A1E002BF9D1704710B4002351
S11301301400621E002C06D003780C781B1B491C8B
S1130140401C002BF4D0180010BC704700E0401C89
S11301500278002A02D002788A42F8D100787047E7
S113016070B504002079002823D0256B01232A00D0
S113017014F13401607802F0E3F9002801D0012081
S113018018E000202071606A854212D3606AE16938
S1130190081885420DD2E67809E0E0694519012383
S11301A02A0014F13401607802F0CAF9761E022E96
S11301B0F3D2002070BD38B504000D00206B8542D9
S11301C012D02000FFF7CCFF002801D001200CE062
S11301D001232A0014F13401607802F064F9002844
S11301E001D0012001E02563002032BD38B50400B0
S11301F02000FFF7B5FF0500EDB2002D5DD120789A
S1130200032852D1607900284FD0002020634FF496
S11302100072002114F13400FFF780FF552084F8A8
S11302203202AA2084F83302522084F83400522087
S113023084F83500612084F83600412084F83700C2
S1130240722084F81802722084F81902412084F87C
S11302501A02612084F81B02206984F81C022069B8
S113026080B2000A84F81D022069000C84F81E0282
S11302702069000E84F81F02E06884F82002E06818
S113028080B2000A84F82102E068000C84F822029B
S1130290E068000E84F823020123626914F134013A
S11302A0607802F04DF9002060710022002160782E
S11302B002F0A4F9002800D001252800C0B232BD04
S11302C0891E8269921E914201D3002003E0827844
S11302D0C06A02FB01007047F8B504000D00022D4E
S11302E002D3A069854201D3012014E020780128BB
S11302F004D00ED303284AD032D30AE02E0016EBE2
S11303005606606A10EB56212000FFF754FF0028C0
S113031002D05FF0FF30F2BD4FF40070B6FBF0F195
S113032001FB1061081990F83470761C606A10EBB8
S113033056212000FFF73FFF0028EAD14FF4007058
S1130340B6FBF0F101FB1061081990F8340057EA8C
S11303500027E80701D5380901E03805000DDAE780
S1130360606A10EB15212000FFF725FF0028D0D18B
S113037068004FF40071B0FBF1F202FB1102101996
S113038034304178007850EA012080B2C3E7606AD3
S113039010EBD5112000FFF70EFF0028B9D1A800FB
S11303A04FF40071B0FBF1F202FB1102101934306A
S11303B0C1788278120452EA0161427851EA02213A
S11303C00078084300010009A5E7F8B504000D0012
S11303D01600022D02D3A069854201D3022082E0D7
S11303E02078012804D07BD3032858D040D377E069
S11303F02F0017EB5707606A10EB57212000FFF717
S1130400DAFEC0B200286CD14FF40070B7FBF0F1F3
S113041001FB1071081910F13401E80705D50878BB
S113042010F00F0050EA061000E0300008707F1C46
S113043001202071606A10EB57212000FFF7BBFEFA
S1130440C0B200284DD14FF40071B7FBF1F202FBAA
S1130450117211193431EA0701D5320906E00A781C
S113046012F0F002330A13F00F031A430A7038E053
S1130470606A10EB15212000FFF79DFEC0B2002832
S11304802FD169004FF40072B1FBF2F303FB121396
S1130490191934310E70B6B2320A4A7021E0606A1A
S11304A010EBD5112000FFF786FEC0B2002818D14A
S11304B0A9004FF40072B1FBF2F303FB12131919F4
S11304C03431CA78120612F0704216430E703200AC
S11304D092B2120A4A70320C8A70320ECA7000E06C
S11304E0022001212171C0B2F2BDF8B504000E0052
S11304F0022E02D3A069864201D3022527E00025FB
S113050009E0206910F1010F04D02069401C20612A
S1130510012060713E00A069864218D2310020009B
S1130520FFF7DAFE0700002F11D0012F01D10225B9
S11305300DE017F1010F01D1012508E0002231007F
S11305402000FFF742FF0500EDB2002DD9D02800AE
S1130550C0B2F2BDF8B504000E00002E07D1E76862
S1130560002F02D0A06987420DD301270BE0310090
S11305702000FFF7B1FE022801D2012043E0A16967
S1130580884240D337003D006D1CA069854204D3E6
S11305900225AF4201D2002035E029002000FFF7F8
S11305A09BFE00281DD17FF0704229002000FFF738
S11305B00CFFC0B2002806D1002E04D02A0031005E
S11305C02000FFF702FFC0B2002814D1E5602069C3
S11305D010F1010F16D02069401E206101206071C6
S11305E010E010F1010F01D0012800D10BE0BD4251
S11305F0CAD1002007E0C0B2012802D15FF0FF3564
S113060000E001252800F2BD70B504000D00E5806E
S1130610A068012803D021688969884201D3022097
S113062048E0002805D121680978032901D1206810
S1130630806A00280ED1E06020680089ADB285424E
S113064001D3022036E02068806AADB210EB1510A9
S1130650206123E02168897889B20E0100E0AD1B96
S1130660ADB2B6B2B54210D301002068FFF734FE34
S113067010F1010F01D101201CE0022803D32168ED
S113068089698842EBD3022014E0E060010020680D
S1130690FFF716FEADB210EB15102061ADB21020BD
S11306A0B5FBF0F101FB1051206810EB4110343020
S11306B06061002070BDF8B504000D00E088461CA0
S11306C0B6B2002E02D02069002801D1042087E0B0
S11306D0B6B21020B6FBF0F101FB1061002972D113
S11306E02069401C2061E068002806D12068008948
S11306F0B6B2864267D3042072E0B6B2206880782E
S1130700401E10EA161F5ED1E1682068FFF7E4FD81
S11307100700022F01D2022062E017F1010F01D17C
S113072001205DE020688069874246D3002D01D115
S1130730042055E0E1682068FFF70CFF0700002F54
S113074001D107204CE0012F01D1022048E017F12C
S1130750010F01D1012043E02068FFF701FD0028CB
S113076001D001203CE04FF40072002120683430B5
S1130770FFF7D4FC39002068FFF7A2FD2168086365
S1130780002505E02068006B401C216808636D1C8F
S113079020688078EDB2854209D220680121017178
S11307A02068FFF7DDFC0028ECD0012018E0206869
S11307B0006BEDB2401B21680863E76039002068D4
S11307C0FFF77EFD2061E680B6B21020B6FBF0F1A3
S11307D001FB1061206810EB41103430606100208F
S11307E0F2BD70B504000D0000212000FFF70CFFDE
S11307F0C0B200281BD1002621692068FFF7DBFC6A
S1130800C0B2002813D161690978E52903D0616970
S11308100978002903D1761CAE4201D107E00026F5
S113082001212000FFF747FFC0B20028E4D0C0B286
S113083070BDCA7E8B7E53EA022292B200780328EE
S113084006D1487D097D51EA002080B252EA004277
S11308501000704781760A0092B2120AC2760A0C1E
S11308600275090C89B2090A417570472DE9F041F6
S113087004000D00287830F04000401E0D2101FBDB
S113088000F600275FF00108DFF8180D385C401906
S11308904078DFF8101D795C495D51EA00201FFAA9
S11308A088F8B8F1000F11D080B202F00CF880463D
S11308B0FF2E09D234F8160002F005F8761C1FFA50
S11308C088F880B2804508D0002018E080B24FF646
S11308D0FF71884201D0002011E07F1C0D2FD3D37B
S11308E0287840060AD51FFA88F8B8F1000F05D019
S11308F034F81600002801D0002000E00120BDE8F3
S1130900F08170B40A7812F03F02521E0D235A434C
S113091000230124DFF88C5C5D5D6D186D78DFF8D1
S1130920846C9E5D765C56EA0525A4B2002C11D039
S1130930FF2A01D3002018E02C0020F81240521C9A
S11309405B1C0D2BE6D3097849060DD5FF2A08D385
S113095000200AE0ADB24FF6FF76B542F0D0002099
S113096003E0002120F81210012070BC7047F0B49D
S11309704B730F23CB7200230B7300238B7600235E
S1130980CB76D2B2531E0D24634300242500A4B2B7
S1130990ADB24FF6FF76B54202D030F813505B1C6F
S11309A0DFF8006CA65D7554DFF8F86BA65D761869
S11309B0ADB22F0A7770ADB2002D01D14FF6FF759D
S11309C0641C0D2CE4D3ADB24FF6FF74A54203D0E2
S11309D030F81300002801D152F040020A70F0BC34
S11309E070477CB5040016001D000B222000FFF7A1
S11309F08BFBADB2062D09DBADB2E80310EB55005D
S1130A0031880D18B61C30880028F5D10720ADB206
S1130A10102195FBF1F202FB115212F13001C9B21F
S1130A203A2900DBC91D00AA8154401EADB2102131
S1130A3095FBF1F5ADB2002DE9D100A97E22425417
S1130A40002100E0491C814202D20A5D202AF9D12A
S1130A500A00511C082803D200ABC35C401C00E010
S1130A60202313550829F3D373BD00210B22C9B2E7
S1130A70CB0113EB510103785918401C521E002A74
S1130A80F5D10800C0B270472DE9F04105000021FE
S1130A902800FFF7B9FD0400E4B2002C02D02000C6
S1130AA0C0B226E0FF27B84629692868FFF783FB10
S1130AB00400E4B2002C1AD16E693078C0B2002868
S1130AC001D1042413E0F17A11F03F01C0B2E5280A
S1130AD004D00A070FD5C9B20F290CD0FF27002173
S1130AE02800FFF7E8FD0400E4B2002CDCD020006D
S1130AF0C0B2BDE8F081C9B20F291ED1E96900294D
S1130B00EDD0410606D596F80D8010F0BF00070021
S1130B10E9882984C0B2FFB2B8420CD1707B5FFA75
S1130B2088F8804507D13100E869FFF79FFE002867
S1130B3001D07F1E00E0FF27D1E7FFB2002F06D1CE
S1130B403000FFF792FF5FFA88F88045CFD0FF2787
S1130B504FF6FF702884A869C07AC007BFD40B225F
S1130B60A9693000FFF7E2FA0028B8D1BFE72DE900
S1130B70F04104000D00FF26FF275FF00408206900
S1130B8000282ED021692068FFF715FB80465FFA04
S1130B9088F8B8F1000F24D160690278D2B2002A33
S1130BA002D15FF004081CE0C17A11F03F01D2B217
S1130BB0E52A0BD0D2B22E2A08D0C9B2082901D115
S1130BC0012300E00023DBB2AB4215D0FF26002155
S1130BD02000FFF770FD80465FFA88F8B8F1000F37
S1130BE0CDD05FFA88F8B8F1000F01D00020206161
S1130BF04046C0B2BDE8F081C9B20F2919D15106EF
S1130C0005D5477B12F0BF021600E1882184D2B2D9
S1130C10F6B2B2420BD1417BFFB28F4207D1010041
S1130C20E069FFF76EFE002801D0761E00E0FF2683
S1130C30CDE7F6B2002E04D1FFF717FFFFB28742CB
S1130C4002D04FF6FF702084CBE72DE9F04184B049
S1130C500400A669E7690C22310000A8FFF754FAE2
S1130C609DF80B00C0072CD50020F0720020E06135
S1130C705FF0010801E018F101081FFA88F8B8F1E3
S1130C80640F0DDA43469BB23A0000A93000FFF727
S1130C90A8FE2000FFF7F8FE0500EDB2002DEAD013
S1130CA01FFA88F8B8F1640F01D107207DE0EDB296
S1130CB0042D02D02800C0B277E09DF80B00F0723A
S1130CC0E7619DF80B00800712D55FF0000801E092
S1130CD018F101081FFA88F837F818000028F7D12E
S1130CE01FFA88F818F119000D2190FBF1F600E0C5
S1130CF00126B6B231002000FFF773FD0500EDB206
S1130D00002D32D1761E300080B200282DD0E0882C
S1130D10811B89B22000FFF777FC0500EDB2002D9E
S1130D2023D1A069FFF7A1FE070021692068FFF71E
S1130D3042FA0500EDB2002D17D13B00DBB23200C0
S1130D40D2B26169E069FFF712FE206801210171E6
S1130D5000212000FFF7AFFC0500EDB2002D04D107
S1130D60761E300080B20028DFD1EDB2002D1AD1FA
S1130D7021692068FFF71FFA0500EDB2002D12D19A
S1130D80202200216069FFF7C9F90B22A16960697B
S1130D90FFF7BAF9A069C07A10F018006169087306
S1130DA02068012101712800C0B204B0BDE8F081BF
S1130DB038B50400E588208C4FF6FF71884201D1D4
S1130DC0290000E0218C89B22000FFF71DFCC0B28D
S1130DD000281BD121692068FFF7EDF9C0B2002873
S1130DE010D16169E5220A70216801220A71E18843
S1130DF0ADB2A94206D200212000FFF75CFCC0B2CC
S1130E000028E7D0C0B2042800D10220C0B232BD0D
S1130E102DE9F14F8846D8F8009001E019F1010955
S1130E2099F800002F28F9D099F800005C28F5D033
S1130E300098C6690024250002E026F815706D1C90
S1130E4014F80970641CBFB2202F05DBBFB22F2F2A
S1130E5002D0BFB25C2F09D114EB0900C8F800001E
S1130E60BFB2202F1FDA5FF004081EE0FF2D01D36C
S1130E70062090E0FFB20121380080B201F0FCFCB2
S1130E800700BFB2002F01D1062084E0BFB2802F3B
S1130E90D3DABFB23900DFF8F808FFF757F90028B2
S1130EA0CBD0062077E05FF0000800E06D1E002D37
S1130EB009D016EB450030F8027CBFB2202FF5D0E4
S1130EC0BFB22E2FF2D0002D01D1062063E0002006
S1130ED026F815000B22202100988069FFF71EF9DF
S1130EE0002400E0641C36F814002028FAD036F8F8
S1130EF014002E28F6D0002C03D058F0030800E08C
S1130F006D1E002D05D016EB450030F8020C2E287E
S1130F10F6D15FF00009CB465FF0080A01E058F013
S1130F20030836F81470641CBFB2002F35D1009842
S1130F3080690078E52803D1009880690521017053
S1130F40BAF1080F01D15FEA89095FFA89F919F04A
S1130F500C000C2805D05FFA89F919F00300032866
S1130F6001D158F002085FEA88700FD45FFA89F95A
S1130F7019F00300012801D158F010085FFA89F92B
S1130F8019F00C00042801D158F008080098806971
S1130F9080F80B800020BDE8F28FBFB2202FBED0B6
S1130FA0BFB22E2F01D1AC42B9D1D34501D2AC424C
S1130FB013D1BAF10B0F02D158F00308B7E7AC42D2
S1130FC001D058F00308A542B1D32C005FF0080B00
S1130FD05FF00B0A5FEA8909A3E7BFB2802F10DB39
S1130FE00021380080B201F047FC0700BFB2002F97
S1130FF005D0BFB2DFF89C07381810F8807C58F091
S11310000208BFB2002F07D0BFB23900DFF888074B
S1131010FFF79CF8002803D05F2758F003080FE07F
S1131020BFB2B7F141001A2802D259F0020907E011
S1131030BFB2B7F161001A2802D259F00109203F6A
S1131040009880690BF800701BF1010B69E7F8B593
S11310500C0004F209010269002A48D04269137B9A
S113106000250EE0F6B2052E00D1E5261F0705D5B2
S1131070F6B2B6F141071A2F00D220360E70491C81
S11310806D1C082D03D2AE5CF6B2202EEAD1157A7F
S1131090202D15D02E250D70491C08250AE0DF06E9
S11310A005D5F6B2B6F141071A2F00D220360E70DC
S11310B0491C6D1C0B2D03D2AE5CF6B2202EEED172
S11310C0D37A2372D37F957F2D0455EA0363557F2A
S11310D053EA0523157F2B432360537E157E55EA7F
S11310E00323A380D37D927D52EA0322E28000226F
S11310F00A70A169002926D0E169002923D0A669D4
S11311000025016900291CD0018C4FF6FF72914221
S113111017D0C76901E0A8556D1C3888BF1C0100B1
S113112089B200290DD0002180B201F0A5FB80B264
S1131130002801D1002504E0E169491E8D42EAD36B
S113114000250020A855F1BD13B5040001980078CE
S11311502F2803D0019800785C2802D10198401C04
S113116001900020A0600198007820280AD2002174
S11311702000FFF749FA0021616120E02068FFF7B1
S113118058FBA06001A92000FFF742FEC0B200286E
S113119015D12000FFF778FCA169C97AC0B20028F4
S11311A006D0C0B204280AD1490700D4052006E0BD
S11311B0490704D46169C87AC006DFD40520C0B2E7
S11311C016BD10B5040001230A0014F1340160783F
S11311D001F069F9002801D003202DE094F83302CE
S11311E094F8321251EA002080B24AF6552188421E
S11311F001D0022020E094F86C0094F86B100902EE
S113120051EA004094F86A100843DFF8781C8842D9
S113121001D1002010E094F8880094F887100902A6
S113122051EA004094F886100843DFF8581C8842BD
S113123001D1002000E0012010BDF8B515000268BE
S11312401378B3F130060A2E05D253783A2B02D123
S1131250921C026000E0002600200860002E01D0ED
S11312600B209DE1DFF8200C50F82640002C01D122
S11312700C2095E10C60207800280DD0607801F0F6
S113128009F9C10708D4EDB2002D03D0400701D5F8
S11312900A2085E1002083E10020207066706078D8
S11312A001F055F8C10701D5032079E1EDB2002D15
S11312B003D0400701D50A2072E10025290020004F
S11312C0FFF77FFF0600F6B2012E1CD10020C0B24A
S11312D0002800D0401EC0B214EB001000F2F2103F
S11312E0017900290FD0C17A827A120452EA01618D
S11312F0427A51EA0221007A50EA010529002000CD
S1131300FFF75FFF0600F6B2032E01D1012047E18B
S1131310F6B2002E01D00D2042E194F8400094F87A
S11313203F1051EA002080B2B0F5007F01D00D20BB
S113133036E194F84B0094F84A1051EA002080B248
S113134000280DD194F85B0094F85A10090451EA6E
S1131350006094F8591050EA012094F8581008439A
S1131360E06194F84410E170C9B2012904D0C9B213
S1131370022901D00D2013E1C9B2484394F8411069
S1131380A170C9B2002903D04A1EC9B2114201D0CA
S11313900D2005E194F8461094F8452052EA012105
S11313A0218121891022B1FBF2F303FB1213002BDC
S11313B001D00D20F4E094F8481094F8472052EA44
S11313C0012292B2002A0DD194F8571094F85620B5
S11313D0120452EA016194F8552051EA022194F86A
S11313E054200A4394F8431094F8423053EA0121FC
S11313F089B2002901D10D20D2E089B2431826898F
S113140013EB16139A4201D20D20C9E0D21AA67822
S1131410B2FBF6F2002A01D10D20C1E0012640F60C
S1131420F677BA4200D302264FF6F677BA4200D3D3
S11314300326921CA261256289B249196162591975
S1131440E162F6B2032E16D12089002801D00D20C6
S1131450A6E094F8630094F86210090451EA00606D
S113146094F8611050EA012094F860100843A062D7
S1131470A069800015E02189002901D10D208FE0A9
S1131480616A4018A062F6B2022E02D1A06940003F
S113149007E0A06903214843217E11F0010111EB0B
S11314A05000E16900F2FF10B1EB502F01D20D2082
S11314B076E05FF0FF3020610020E060F6B2032E9A
S11314C060D10020607194F8650094F8641051EACA
S11314D0002080B2401960610123626914F1340173
S11314E0607800F0E0FF00284CD194F8330294F8BF
S11314F0321251EA002080B24AF65521884241D185
S113150094F8370094F83610090451EA006094F80E
S1131510351050EA012094F834100843DFF8381AE3
S113152088422FD194F81B0294F81A12090451EA44
S1131530006094F8191250EA012094F81812084334
S1131540DFF8181A88421DD194F8230294F8221265
S1131550090451EA006094F8211250EA012094F839
S113156020120843E06094F81F0294F81E12090444
S113157051EA006094F81D1250EA012094F81C12FC
S1131580084320612670DFF8D8090088401CDFF882
S1131590D0190880E0800020206300202071002002
S11315A0F2BD0000D85A000080B500280BD00168B5
S11315B0002908D001680978002904D00168C98885
S11315C08288914201D0092008E00068407800F048
S11315D061FFC00701D5032000E0002002BDC0B2B6
S11315E0002801D00B2012E0C0B2DFF89C2852F88A
S11315F02020002A01D000231370002901D00022EA
S11316000A70C0B2DFF8802842F82010002070472A
S11316102DE9F2438CB004001500002C01D10920FF
S1131620B3E00020206015F01F0515F0FE0200A9AC
S11316300CA8FFF702FE0600F6B2002E40F0A380CD
S113164009A80690DFF81C0907900C9900A8FFF779
S11316507BFD0600059FF6B2002E02D1002F00D1BB
S113166006261C20054258D0F6B2002E0AD0F6B247
S1131670042E03D100A8FFF7E8FA060055F0080588
S1131680059F08E0F87A1121084201D0072602E0FC
S1131690680700D50826F6B2002E4CD128074AD593
S11316A001F0D1F8804687F80E80404680B2000AE7
S11316B0F8735FEA184038745FEA186078740020A1
S11316C0F87200203877002078770020B87700205F
S11316D0F87739000098FFF7ACF88146002138000C
S11316E0FFF7B8F8009801210171B9F1000F22D079
S11316F00098D0F8308049460098FEF7F6FE0600C0
S1131700F6B2002E17D10098B9F10101C16041462B
S11317100098FEF750FD06000DE0F6B2002E0AD147
S1131720F87AC00601D5042605E0A80703D5F87A9F
S1131730C00700D50726F6B2002E07D1280701D529
S113174055F020050098006BE0612762F6B2002E88
S113175019D1A57139000098FFF76BF82061F87F63
S1131760B97F090451EA0060797F50EA0120397F8A
S11317700843E0600020A0600020A0610098206081
S11317800098C088A0803000C0B20DB0BDE8F083DE
S1131790185B0000A8550000485B00002DE9F047E5
S11317A0050016001F000C00002038602800FFF719
S11317B0FBFEC0B2002801D0C0B2E7E0A879000661
S11317C001D50220E2E0A879C00701D40720DDE0BA
S11317D0E868A968401AB04229D2060027E0C5F893
S11317E01890A8684FF40071B0FBF1F202FB1102EB
S11317F0D2F50078464500D2B0464246A8684FF478
S11318000071B0FBF1F303FB1103581910F124012B
S11318102000FEF779FC18EB0404A86818EB00001C
S1131820A860386818EB00003860B6EB0806002E94
S113183000F0AB80A8684FF40071B0FBF1F202FB3A
S11318401102002ACDD1A868400A29688978491E66
S113185011EA00085FFA88F8B8F1000F1AD1A868F5
S1131860002801D1286903E069692868FEF734FD7E
S1131870022805D2A87950F08000A871022085E0E2
S113188010F1010F05D1A87950F08000A871012052
S11318907CE0686169692868FEF712FD8146B9F148
S11318A0000F05D1A87950F08000A87102206DE0E6
S11318B05FFA88F818EB09095FEA562ABAF1000FB3
S11318C037D0286880785FFA88F81AEB08018842D4
S11318D005D2286880785FFA88F8B0EB080A534686
S11318E0DBB24A4621002868407800F0DCFD00287D
S11318F005D0A87950F08000A871012046E0A879AD
S1131900400611D5A869B0EB090050450CD24FF43C
S1131910007215F12401A869B0EB09004FF40073BB
S113192003FB0040FEF7F0FB4FF4007000FB0AF8E5
S113193071E7A86948453FF452AFA879400613D52A
S11319400123AA6915F124012868407800F0F8FD04
S1131950002805D0A87950F08000A871012015E076
S1131960A87910F0BF00A87101234A4615F124019B
S11319702868407800F097FD00283FF430AFA8793C
S113198050F08000A871012000E00020BDE8F0873D
S11319902DE9F047050016001F000C0000203860F8
S11319A02800FFF701FEC0B2002801D0C0B270E0E9
S11319B0A879000601D502206BE0A879800701D43C
S11319C0072066E0E8683018E96888422DD20026CE
S11319D02BE0C5F81890A8684FF40071B0FBF1F241
S11319E002FB1102D2F50078464500D2B0464246C9
S11319F02100A8684FF40073B0FBF3FC0CFB130C3C
S1131A001CEB05002430FEF77FFBA87950F0400062
S1131A10A87118EB0404A86818EB0000A8603868E3
S1131A2018EB00003860B6EB0806002E26D0A86834
S1131A304FF40071B0FBF1F202FB1102002ACAD18B
S1131A40A868400A29688978491E11EA00085FFAE3
S1131A5088F8B8F1000F30D1A868002808D12869A7
S1131A60002809D100212868FEF774FD286103E0ED
S1131A7069692868FEF76EFD00280CD1E868A9683A
S1131A80884201D2A868E860A87950F02000A871C3
S1131A900020BDE8F087012805D1A87950F0800026
S1131AA0A8710220F5E710F1010F05D1A87950F0D3
S1131AB08000A8710120ECE76861A879400613D57D
S1131AC00123AA6915F124012868407800F038FD43
S1131AD0002805D0A87950F08000A8710120D8E72B
S1131AE0A87910F0BF00A87169692868FEF7E8FBBF
S1131AF08146B9F1000F05D1A87950F08000A87192
S1131B000220C6E75FFA88F818EB09095FEA562A4B
S1131B10BAF1000F38D0286880785FFA88F81AEB99
S1131B200801884205D2286880785FFA88F8B0EB0B
S1131B30080A5346DBB24A4621002868407800F080
S1131B40FFFC002805D0A87950F08000A87101207E
S1131B509FE7A869B0EB0900504510D24FF400721A
S1131B60A869B0EB09004FF4007101FB004115F1C5
S1131B702400FEF7C9FAA87910F0BF00A8714FF449
S1131B80007000FB0AF844E7A86948453FF421AF18
S1131B90A868E9688842BFF41CAF01234A4615F1DE
S1131BA024012868407800F07EFC00283FF411AF3F
S1131BB0A87950F08000A87101206AE738B50400C4
S1131BC02000FFF7F1FCC0B200284AD1A1798906B0
S1131BD047D5A07940060FD50123A26914F1240149
S1131BE02068407800F0ACFC002801D0012039E0E6
S1131BF0A07910F0BF00A071E1692068FEF7DBFA5C
S1131C00C0B200282DD1256AE87A50F02000E8728D
S1131C10E0682877E06880B2000A6877E068000C22
S1131C20A877E068000EE87721692800FEF712FE25
S1131C3000F009FEA875010089B2090AE975010CD2
S1131C402976000E68760020A8740020E874A07934
S1131C5010F0DF00A0712068012101712068FEF7F7
S1131C60C5FAC0B232BD10B504002000FFF7A6FFCC
S1131C70C0B2002801D100212160C0B210BD2DE9FD
S1131C80F04104000D002000FFF78EFC0600F6B2C0
S1131C90002E02D03000C0B2CCE0A079000601D5FD
S1131CA00220C7E0E068A84203D2A079800700D4EC
S1131CB0E568A0680027A760002D7BD0216889789B
S1131CC04FF4007202FB01F8002810D0411EB1FB52
S1131CD0F8F16A1EB2FBF8F28A4208D3401EB8F14A
S1131CE001018843A060A0682D1A606919E0206989
S1131CF0002815D100212068FEF72CFC012805D10D
S1131D00A07950F08000A071022093E010F1010F3F
S1131D1005D1A07950F08000A07101208AE02061F3
S1131D206061002807D145E06061A16818EB0101FA
S1131D30A160B5EB0805A84509D2A17989071ED58C
S1131D4001002068FEF706FC00281CD14546A16866
S1131D506918A1604FF40071B5FBF1F202FB115256
S1131D60002A27D001002068FEF7AAFA0700002FF6
S1131D701ED1A07950F08000A07102205AE0010029
S1131D802068FEF7A9FA10F1010F05D1A07950F0EF
S1131D908000A07101204DE0022803D321688969E5
S1131DA08842C1D3A07950F08000A071022041E0A4
S1131DB017EB5527A0684FF40071B0FBF1F202FB5A
S1131DC01102002A2AD0A069874227D0A0794006B0
S1131DD013D50123A26914F124012068407800F08E
S1131DE0AFFB002805D0A07950F08000A07101203D
S1131DF020E0A07910F0BF00A07101233A0014F193
S1131E0024012068407800F04EFB002805D0A0791A
S1131E1050F08000A07101200CE0A761E068A16887
S1131E20884205D2A068E060A07950F02000A0713B
S1131E303000C0B2BDE8F08131B58CB00C00002296
S1131E4003A90CA8FFF7F9F90500EDB2002D15D18F
S1131E5000A80990DFF80C010A900C9903A8FFF779
S1131E6073F90500EDB2002D08D10898002804D0BC
S1131E70210003A8FFF7EBF800E006252800C0B214
S1131E800DB030BD46415400340F002071B595B0FB
S1131E90012200A915A8FFF7D0F90400E4B2002C30
S1131EA056D109A806902F480790159900A8FFF766
S1131EB04BF90400E4B2002C4AD1059D002D01D158
S1131EC0062403E0E87AC00700D507242900009817
S1131ED0FEF7AFFC0600E4B2002C21D1E87AC0067C
S1131EE01ED5022E01D202241AE0242200A90CA835
S1131EF0FEF70AF90E9602210CA8FEF785FB0400F2
S1131F00E4B2002C0CD100210CA8FEF730FE040032
S1131F10E4B2002C00D10724E4B2042C00D1002444
S1131F20E4B2002C14D100A8FEF742FF0400E4B28E
S1131F30002C0DD1002E04D031000098FEF7D5FA04
S1131F400400E4B2002C03D10098FEF74FF904001A
S1131F502000C0B216B070BD52526141727241612C
S1131F60400F00208C0A00202DE9FC4104000F00E2
S1131F70904600252600FFE7781E854213DA00AB61
S1131F80012201A94046FFF709FC009801280AD163
S1131F909DF80400C0B20D28EED03070761C6D1C84
S1131FA0C0B20A28E8D100203070002D00D10024EE
S1131FB02000BDE8F68130B583B004000D00E4B222
S1131FC00A2C03D129000D20FFF7F5FF8DF80040FE
S1131FD0012401AB220000A92800FFF7D9FC0198D5
S1131FE0A04201D1012001E05FF0FF303EBD70B599
S1131FF004000D00002601E0641C761C20780028F3
S113200009D029002078FFF7D6FF10F1010FF3D192
S11320105FF0FF3000E0300070BD10B450F8041BD6
S113202081B102681218001D50F8043BDC0744BF5C
S1132030A9F10104E31852F8044B43F8044B091FB7
S1132040F9D1EBE710BC704710B582B00122012131
S1132050DFF8F80700F0A9FD20215FF0402000F030
S1132060B8FD202220215FF0402000F09EFD0024D6
S11320700AE0FF21DFF8D80700F0E0FE00A9DFF84E
S1132080D00700F0FAFE641C0A2CF2D320215FF082
S1132090402000F0CBFD13BD00B583B0DFF8B407DA
S11320A001F05CF8DFF8B00701F058F8DFF8AC078E
S11320B001F054F834215FF0402000F0B7FD012115
S11320C0DFF8880700F085FD0A23022234215FF03F
S11320D0402000F0B7FC0A2302220121DFF86C073C
S11320E000F0B0FC01220121DFF8600700F05DFD83
S11320F001F0B2F908210191DFF86417009100237F
S113210000220100DFF8480700F0FDFDDFF840077A
S113211000F072FEFFF798FF07BD1CB5DFF830072B
S113212000F07BFE01F098F94408DFF83807844298
S113213001D3DFF8344701F08FF9082101910094AD
S1132140002300220100DFF8080700F0DCFDDFF8BF
S1132150000700F051FE13BDDFF81007007850F0BF
S11321600100DFF808170870704780B5C0B201009D
S1132170DFF8DC0600F062FE00A9DFF8D40600F008
S11321807CFE0098C0B202BD10B50400FF20FFF72A
S1132190ECFF207010BD38B501F0ADFA10F5FA75FA
S11321A0FF20FFF7E2FF0400E4B2FF2C03D001F0AC
S11321B0A2FAA842F4D3E4B2FF2C01D1012000E03A
S11321C0002032BD80B501220121DFF8800600F035
S11321D0ECFCFF20FFF7C9FF01BD80B500220121FF
S11321E0DFF8680600F0E1FCFF20FFF7BEFFFFF711
S11321F0D2FF002801D0012002E0FFF7E3FF002016
S113220002BDF8B504000D0001F075FA10F1640781
S1132210FF20FFF7AAFF0600F6B2FF2E03D101F05C
S11322206AFAB842F4D3F6B2FE2E01D0002011E0CF
S11322302000FFF7A9FF641C2000FFF7A5FF641C22
S1132240AD1E002DF4D1FF20FFF78FFFFF20FFF715
S11322508CFF0120F2BD38B504000D00FFF79BFF91
S1132260002801D1002024E02800C0B2FFF77DFF40
S1132270EDB2FD2D1CD04FF400752078FFF775FFEB
S1132280641C2078FFF771FF641CAD1E002DF4D18F
S1132290FF20FFF76AFFFF20FFF767FFFF20FFF72C
S11322A064FFC0B210F01F00052801D0002000E038
S11322B0012032BD38B504000D0020060AD514F003
S11322C07F0400213720FFF7F5FFC0B2022801DBAD
S11322D0C0B23BE0FFF776FFFFF77FFF002801D194
S11322E0FF2033E054F04000C0B2FFF73EFF280E59
S11322F0C0B2FFF73AFF280CC0B2FFF736FF280A36
S1132300C0B2FFF732FF2800C0B2FFF72EFF01254D
S1132310E4B2002C00D19525E4B2082C00D1872525
S11323202800C0B2FFF721FFE4B20C2C02D1FF2039
S1132330FFF71BFF0A25FF20FFF717FF010604D54F
S11323406D1E2900C9B20029F5D1C0B232BD70B5E5
S113235082B0C0B2002801D001209AE0DFF80C0559
S11323600078800703D5DFF80405007891E0FFF7D3
S113237093FE00220121DFF8D40400F016FC0025AE
S113238000210020FFF796FF012869D101F0B3F97D
S113239010F57A764FF4D5710820FFF78BFF0128EA
S11323A03CD1002406E0FF20FFF7DFFEE4B200A9E1
S11323B06054641CE4B2042CF5DB9DF8020001288F
S11323C04ED19DF80300AA284AD101F094F9B042F5
S11323D006D25FF08041A920FFF76CFF0028F4D1FA
S11323E001F089F9B0423BD200213A20FFF762FFA5
S11323F0002835D1002406E0FF20FFF7B6FEE4B242
S113240000A96054641CE4B2042CF5DB9DF80000C0
S1132410400601D50C2500E0042521E00021A92077
S1132420FFF748FF022802DA0225A92401E001256A
S1132430012401F060F9B04206D200212000C0B2AC
S1132440FFF738FF0028F4D101F055F9B04206D265
S11324504FF400711020FFF72DFF002800D0002555
S1132460DFF80C04EDB20560FFF7ACFEEDB2002D11
S11324700AD0DFF8F803007810F0FE00DFF8EC1360
S11324800870FFF74AFE01E0FFF766FEDFF8DC03A1
S1132490007876BDC0B2002801D0012002E0DFF848
S11324A0CC030078704738B50C0011001D00C0B291
S11324B0002802D1EDB2002D01D104203FE0DFF865
S11324C0AC030078C00701D5032038E0DFF8A0038F
S11324D00078000702D44FF400704143EDB2012D9F
S11324E00DD11120FFF7E6FE00281FD14FF4007133
S11324F02000FFF786FE002818D0002516E01220E1
S1132500FFF7D8FE002811D14FF400712000FFF727
S113251078FE002806D014F500746D1E2800C0B2A1
S11325200028F1D100210C20FFF7C4FEFFF74AFE7A
S1132530EDB2002D01D0012000E00020C0B232BD78
S113254070B50C0015001E00C0B2002802D1F6B20E
S1132550002E01D1042050E0C4480078C00701D502
S113256003204AE0C1480078400701D5022044E036
S1132570BF480078000702D44FF400704543F6B218
S1132580012E0DD129001820FFF794FE00282BD12D
S1132590FE212000FFF75FFE002825D0002623E05F
S11325A0B348007810F0060F04D0F6B2310097203B
S11325B0FFF780FE29001920FFF77CFE002813D1C5
S11325C0FC212000FFF747FE002806D014F5007414
S11325D0761E3000C0B20028F2D1FD210020FFF7A2
S11325E03AFE002800D10126FFF7ECFDF6B2002EDA
S11325F001D0012000E00020C0B270BD30B585B02C
S113260014002200C0B2002801D0042019E1974828
S11326100078C00701D5032013E10125C9B20029C0
S113262013D0012917D003295ED00A2900F0BB80FA
S11326300B2900F0BD800C2900F0C8800D2900F0A2
S1132640D3800E2900F0E380F6E0FFF7C6FD0028F2
S113265000D00025F1E000210920FFF72BFE00281F
S113266041D1102100A8FFF7CCFD00283BD09DF8F4
S11326700000C0B28009C0B201280FD19DF8090042
S11326809DF8081010EB01209DF8071011F03F0190
S113269010EB0140401C8002206023E09DF80500FF
S11326A010F00F009DF80A10C9B210EBD1109DF87C
S11326B0091011F0030110EB4100851C9DF808007E
S11326C0C0B28009C0B29DF8071010EB81009DF8DC
S11326D0061011F0030110EB8120401CB5F1090133
S11326E0884020600025A8E061480078400720D594
S11326F000218D20FFF7DEFD002853D1FF20FFF7D6
S113270034FD102100A8FFF77CFD00284AD03025B5
S113271003E0FF20FFF729FD6D1EEDB2002DF8D177
S113272010209DF80A10C9B20909884020600025CC
S113273038E000210920FFF7BDFD002832D1102127
S113274000A8FFF75EFD00282CD0494800788007D8
S113275013D59DF80A0010F03F009DF80B10C9B284
S1132760C909C9B211EB4000401C9DF80D10C9B253
S11327708909491E8840206013E09DF80A00C0F3CF
S11327808400C0B2401C9DF80B1011F003019DF8A9
S11327900B20D2B25209D2B212EBC101491C4843F8
S11327A02060002549E0324800681070002544E0AC
S11327B000210920FFF77EFD002806D1102120000A
S11327C0FFF71FFD002800D0002536E000210A2075
S11327D0FFF770FD002806D110212000FFF711FD3E
S11327E0002800D0002528E000213A20FFF762FDF0
S11327F000280BD1002505E0FF20FFF7B6FCEDB261
S113280028556D1CEDB2042DF6DB002515E01848A3
S1132810007840070FD500218D20FFF74BFD0028DD
S113282009D1FF20FFF7A1FC40212000FFF7E9FCBC
S1132830002800D0002500E00425FFF7C3FC280091
S1132840C0B205B030BD0B487047000000700040B6
S1132850008000401000001001000020080000204B
S1132860801A060021BCBE0020BCBE00000000206F
S1132870380F00200000AA4280B2802801DA01004B
S11328801EE000290CD080B2FF2801DD002106E003
S113289080B2194911EB4000B0F5807001880FE057
S11328A0002100E0491C89B2802906DA89B2124A63
S11328B032F8112080B29042F4D111F18000C1B2FB
S11328C0080080B27047002100E0491C0B4A32F82E
S11328D01120002A05D0094A32F8112080B2904212
S11328E0F3D1064A32F81120002A03D0044830F804
S11328F01100FFE780B27047DC5300001C50000059
S1132900FC510000B0F1402F5BD0DFF80013884287
S113291057D0DFF8FC12884253D0DFF8F81288420F
S11329204FD0DFF8F41288424BD0DFF8F01288421F
S113293047D0DFF8EC12884243D0DFF8E81288422F
S11329403FD0DFF8E41288423BD0DFF81813884206
S113295037D0DFF81413884233D0DFF810138842DD
S11329602FD0DFF80C1388422BD0DFF808138842ED
S113297027D0DFF80413884223D0DFF800138842FD
S11329801FD0DFF8FC1288421BD0DFF830138842D6
S113299017D0DFF82C13884213D0DFF828138842AD
S11329A00FD0DFF8241388420BD0DFF820138842BD
S11329B007D0DFF81C13884203D0DFF818138842CD
S11329C001D1012000E00020C0B2704770B50400BE
S11329D00D0016002000FFF795FF002805D14FF4E5
S11329E09071DFF8F40200F095FE002E09D0012E5C
S11329F007D0022E05D04FF49171DFF8DC0200F00D
S1132A0089FEF00705D514F580600068EDB228430F
S1132A1004E014F580600068EDB2A84314F5806109
S1132A200860B00705D514F584600068EDB228434A
S1132A3004E014F584600068EDB2A84314F58461E1
S1132A40086070BDF8B504000D0017001E002000DA
S1132A50FFF758FF002805D140F2FF11DFF8780294
S1132A6000F058FE012F0BD0022F09D0042F07D0FD
S1132A700C2F05D040F20321DFF85C0200F04AFE7F
S1132A80082E0DD00A2E0BD00C2E09D0092E07D0FB
S1132A90002E05D04FF40271DFF83C0200F03AFE3C
S1132AA0F80705D514F5A0600068EDB2284304E0EA
S1132AB014F5A0600068EDB2A84314F5A0610860A5
S1132AC0B80704D5D4F80405EDB2284303E0D4F8DC
S1132AD00405EDB2A843C4F80405780705D514F538
S1132AE0A1600068EDB2284304E014F5A160006819
S1132AF0EDB2A84314F5A1610860380705D514F5B3
S1132B00A3600068EDB2284304E014F5A3600068F4
S1132B10EDB2A84314F5A3610860F00704D5D4F816
S1132B200C05EDB2284303E0D4F80C05EDB2A8433C
S1132B30C4F80C05B00705D514F5A2600068EDB221
S1132B40284304E014F5A2600068EDB2A84314F52C
S1132B50A2610860700704D5D4F81405EDB22843C7
S1132B6003E0D4F81405EDB2A843C4F81405300703
S1132B7004D5D4F81C05EDB2284303E0D4F81C05B1
S1132B80EDB2A843C4F81C05002E05D114F5A560C8
S1132B900068EDB2284304E014F5A5600068EDB2C6
S1132BA0A84314F5A5610860F1BD70B504000D00DB
S1132BB016002000FFF7A6FE002805D140F285315B
S1132BC0DFF8140100F0A6FDEDB2F6B244F825607A
S1132BD070BD38B504000D002000FFF793FE0028F7
S1132BE005D140F2F141DFF8F00000F093FD082335
S1132BF001222900C9B22000FFF724FF0122290085
S1132C00C9B22000FFF7E2FE31BD0000008005409C
S1132C1000500040009005400060004000A00540C6
S1132C200070004000B005400040024038B5040088
S1132C300D002000FFF766FE002804D140F29661E3
S1132C40254800F067FD02222900C9B22000FFF7E1
S1132C50BDFE082301222900C9B22000FFF7F2FEBD
S1132C6031BD000000C005400050024000D00540C6
S1132C700060024000E005400070024000F00540A2
S1132C8000D0034038B504000D002000FFF73AFEE1
S1132C90002804D140F2EA610F4800F03BFD022213
S1132CA02900C9B22000FFF791FE08230122290060
S1132CB0C9B22000FFF7C6FE31BD00000000064087
S1132CC00010064000200640003006400040064048
S1132CD00050064000600640B4570000DFF8C01101
S1132CE088420BD0DFF8BC11884207D0DFF8B81156
S1132CF0884203D0DFF8B411884201D1012000E0FA
S1132D000020C0B270472DE9F84304000F001500FD
S1132D1099462000FFF7E2FF002804D1CC21DFF818
S1132D20900100F0F7FC002D0ED0022D0CD0012DE7
S1132D300AD0032D08D0102D06D0202D04D0D22186
S1132D40DFF86C0100F0E6FCB9F1000F0AD0B9F12C
S1132D50010F07D0B9F1020F04D0D521DFF85001DB
S1132D6000F0D8FCDDF82080B9F1000F02D178081A
S1132D7040450BD2B9F1000F04D00C20B7FBF0F0A2
S1132D80404503D2D7214A4800F0C4FCB7FBF8F011
S1132D90B0F57E4F03D9D821454800F0BBFC099E0D
S1132DA0301F0D2803D3D921414800F0B3FCB9F1F9
S1132DB0020F01D1082000E00020B9F1000F01D179
S1132DC0002100E0042108436060B7FBF8F0002113
S1132DD0891CB0FBF1F2521EFF2AF9D8216115F0CB
S1132DE00300800115F0300550EA02202843711ECB
S1132DF008432060BDE8F18310B504002000FFF70C
S1132E006DFF002804D14FF48571294800F082FC3D
S1132E10606850F00200606010BD10B5040020002E
S1132E20FFF75CFF002804D140F22311204800F092
S1132E3071FC606830F00200606010BD38B50400B9
S1132E400D002000FFF74AFF002804D140F223219F
S1132E50174800F05FFC7FF00100216811F00F01BA
S1132E608840054204D040F22521114800F052FC6C
S1132E70E0688007FCD5A56031BD38B504000D00BD
S1132E802000FFF72BFF002804D140F27F210848DF
S1132E9000F040FCE0684007FCD5A068286031BD24
S1132EA0008000400090004000A0004000B00040BE
S1132EB010580000DFF81413884200F04A81DFF84C
S1132EC01013884200F04581DFF80813884200F0AF
S1132ED04081DFF80413884200F03B81DFF8FC12E4
S1132EE0884200F03681DFF8F812884200F0318120
S1132EF0DFF8F012884200F02C81DFF8EC128842EF
S1132F0000F02781DFF8E412884200F02281DFF824
S1132F10E012884200F01D81DFF8D812884200F0E8
S1132F201881DFF8D412884200F01381DFF8CC1244
S1132F30884200F00E81DFF8C812884200F009814F
S1132F40DFF8C012884200F00481DFF8BC12884226
S1132F5000F0FF80DFF8B412884200F0FA80DFF856
S1132F60B012884200F0F580DFF8A812884200F021
S1132F70F080DFF8A412884200F0EB80DFF89C12A6
S1132F80884200F0E680DFF89812884200F0E18081
S1132F90DFF89012884200F0DC80DFF88C1288425F
S1132FA000F0D780DFF88412884200F0D280DFF886
S1132FB08012884200F0CD80DFF87812884200F059
S1132FC0C880DFF87412884200F0C380DFF86C1206
S1132FD0884200F0BE80402800F0BB80B0F1102F82
S1132FE000F0B780DFF85812884200F0B280DFF8B2
S1132FF05412884200F0AD80DFF84C12884200F091
S1133000A880DFF84812884200F0A380DFF8B813E4
S1133010884200F09E80DFF8B413884200F0998063
S1133020DFF8AC13884200F09480DFF8A8138842DC
S113303000F08F80DFF8A013884200F08A80DFF868
S11330409C13884200F08580DFF89413884200F0D6
S11330508080B0F1101F7CD0DFF88813884278D0CC
S1133060DFF88413884274D0DFF88013884270D06C
S1133070DFF87C1388426CD0DFF87813884268D07C
S1133080DFF87413884264D0DFF87013884260D08C
S1133090DFF86C1388425CD0DFF86813884258D09C
S11330A0DFF86413884254D0DFF86013884250D0AC
S11330B0DFF85C1388424CD0DFF85813884248D0BC
S11330C0DFF85413884244D0DFF85013884240D0CC
S11330D0DFF84C1388423CD0DFF84813884238D0DC
S11330E0DFF84413884234D0DFF84013884230D0EC
S11330F0DFF83C1388422CD0DFF83813884228D0FC
S1133100DFF83413884224D0B0F1202F21D0DFF827
S11331102C1388421DD008281BD0DFF824138842C2
S113312017D0DFF82013884213D0DFF81C1388422D
S11331300FD0DFF8181388420BD0DFF8141388423D
S113314007D0DFF81013884203D0DFF8081588424F
S113315001D1012000E00020C0B2704710B5040086
S11331602000FFF7A7FE002805D140F29631DFF8D2
S1133170E00400F0CFFA14F0704010F1805F0DD13C
S1133180C4F30720DFF8D0140818E1B2890051EA2B
S1133190401050F084400121016011E0200FDFF85D
S11331A0BC1451F820000068A1B2220C12F01F02D6
S11331B091400843210FDFF8A42452F8211008603D
S11331C010BD00000138FDD17047704701001000A8
S11331D002001000000110000002100000041000A2
S11331E0000110100002101000041010005800F02C
S11331F00040101000501020005400F00100002086
S1133200020000200400002008000020100000201C
S11332102000002040000020800000200001002049
S1133220090800F00A0800F00B0800F00C0800F090
S11332300D0800F00E0800F00F0800F0100800F070
S113324000400010022000F0032000F0042000F0F1
S113325070B50400DFF81404006810F0E04F08D0E3
S1133260DFF808040068DFF808140840B0F1805F54
S113327002D1002C00F1A780DFF8E4030568DFF831
S1133280F403066855F4006535F4800556F40066C9
S1133290DFF8CC030560DFF8DC030660A80701D57E
S11332A0A00708D515F0010014F0010191F0010107
S11332B0C0B208421ED074F003000540DFF8A0033A
S11332C00560002E07D516F07000302809D016F0DE
S11332D07000702805D0002E08D415F03000302876
S11332E004D14FF48050FFF76DFF03E05FF400203A
S11332F0FFF768FF35F4FE6514F4FE600543DFF85C
S113330078030640DFF874032040064314F00800F5
S113331056EAC006DFF848030560DFF85803066084
S11333201020FFF74FFF35F4405514F44050054387
S113333036F4005614F400500643DFF82803402105
S11333400160002E06D5DFF82C030660DFF81003B9
S1133350056005E0DFF808030560DFF81803066080
S1133360DFF81C030540DFF81C032040054336F05A
S1133370FC5614F0FC500643600008D555F4800553
S113338036F48006DFF800032040064301E036F0FF
S1133390804620050ED44FF4004000E0401E002873
S11333A004D0DFF8C41209684906F7D535F400657E
S11333B036F40066DFF8A8020560DFF8B80206609C
S11333C01020FFF7FFFE70BD052000F00010101064
S11333D000011020004800F080000030005000F090
S11333E010000030014000F0000100100002001045
S11333F01000001020000010021C00F0031C00F05C
S11334002000003001001010020010100400101001
S113341008001010040400F0050400F0010000107E
S11334200200001004000010031800F0041800F05B
S1133430051800F0061800F0071800F0010010202D
S113344000101000005C00F0015C00F0025C00F071
S1133450035C00F0045C00F030B4DFF8040201689F
S1133460DFF810020268002A02D512F0700001E0B1
S113347011F0300000280DD010283AD020286FD049
S1133480302800F0A480602800F0A480702800F0A8
S1133490A480A5E0C1F38410DFF8F03153F82000D4
S11334A0DFF8EC31134013F1004F05D0002A00F18E
S11334B0AA800B0500F1A780DFF8D8311B68DFF87C
S11334C0AC41246814F0E04F09D0DFF8A04124682F
S11334D0DFF89C512C40B4F1805F40F08380C3F34B
S11334E04814A41C604313F01F04A41CB0FBF4F0A4
S11334F081E0DFF87801006810F0E04F08D0DFF8D1
S11335006C010068DFF868311840B0F1805F02D1C7
S1133510DFF8840123E0DFF854010068DFF850315C
S11335201840DFF87831984205D1DFF8400100688F
S113353080B202280ED0DFF834010068DFF83031A1
S11335401840DFF85C31984207D1DFF820010068A9
S1133550000402D1DFF84C0101E0DFF84C019FE7E1
S1133560DFF80801006810F0E04F08D0DFF8FC0035
S11335700068DFF8FC301840B0F1805F02D1DFF85A
S11335802C0123E0DFF8E4000068DFF8E4301840A1
S1133590DFF80831984205D1DFF8D000006880B226
S11335A002280ED0DFF8C4000068DFF8C4301840E9
S11335B0DFF8EC30984207D1DFF8B000006800046F
S11335C002D1DFF8EC0001E0DFF8E80068E747F239
S11335D0305065E75FF4800062E74FF400405FE736
S11335E0002032E0C3F34814604313F01F04641C4A
S11335F06400B0FBF4F05C0400D540081B0400D563
S1133600800851F480014B021FD5002A18D55300BD
S113361010D5DFF87C30134013F1004F03D0002A9B
S113362008D4090506D44000C2F38651491CB0FBF6
S1133630F1F00AE0C2F3C551491CB0FBF1F004E01B
S1133640C1F3C351491CB0FBF1F030BC704700001A
S1133650F4560000055C00F000E60F40305B00000B
S113366060E00F4058E00F4050E00F4000E00F4092
S11336700000FF7070E00F408FFFFF7F300000807C
S1133680FCFF3FF80300C00700004040285600003C
S11336900008008064E00F40C0E1E4000000011075
S11336A000000310001BB7000024F4007038390038
S11336B0C0C62D0000093D0080B500F00EF8114889
S11336C04CF24F3101601048002101600F48052180
S11336D001600F480021016001BD0C480021016018
S11336E070470A480068C00304D509480068401CB4
S11336F007490860704780B5FFF7F3FF0448006886
S113370002BD000014E000E018E000E010E000E07A
S11337103C0F002080B5034A10600348016000F0AC
S113372006F8FCE7280F00202C0F00207047704794
S113373080B5DFF8780600210170DFF874160020E8
S1133740FDF74DFFC0B2002804D07C21DFF86406E9
S1133750FFF7E0FF01BDDFF854060078002801D12F
S1133760012000E00020704780B500F0E5FB01284F
S113377001D1002011E0DFF834060078002801D0E0
S113378000200AE000F0DCFB012805D1DFF81C066C
S113379001210170012000E0002002BD10B5DFF816
S11337A00C060078002800F0FF81DFF8000600789E
S11337B0012834D100F0DEFBDFF8FC0500F007FC43
S11337C0DFF8F80500F003FC00F0D2FB0122010051
S11337D0DFF8EC05FDF71CFF002807D0DFF8E4054F
S11337E000F0F5FB012000F0E8FBDDE1DFF8D8058F
S11337F000F0EDFBDFF8D40500F0E9FBDFF8D005BD
S113380000F0E5FBDFF8CC0500210160DFF8C4051A
S113381000214160DFF8940502210170C4E1DFF862
S11338208C050078022840F0F780DFF894254FF4E7
S11338308071DFF8A405FEF797FBDFF8741591F8A3
S11338403A12C1F3C01111F0010101290FDBDFF8B5
S1133850740500F0BCFB022000F0AFFBDFF860054C
S1133860FEF701FADFF84405002101709CE100280D
S11338701BD00022DFF86415DFF85C0500F0D6F9F0
S1133880040024B214F1010F0FD1DFF8380500F061
S11338909EFB032000F091FBDFF82405FEF7E3F91B
S11338A0DFF80805002101707EE124B2012C28DB39
S11338B0DFF82005406800280BD1DFF81C05D0F89C
S11338C08001DFF810150860DFF8080524B24460B1
S11338D017E0DFF80405D0F88001DFF8F814096870
S11338E0884206D2DFF8F004D0F88001DFF8E4144F
S11338F00860DFF8E004406824B22018DFF8D4142C
S11339004860DFF8AC04D0F83C02DFF8A414D1F826
S11339104012884201D1012000E000200128C0F2B9
S113392043810021DFF89804FEF7A9F900280FD09D
S1133930DFF8900400F04BFB042000F03EFBDFF8BE
S11339408004FEF790F9DFF86404002101702BE194
S1133950DFF8740400F03BFBDFF8840400F037FB6D
S1133960DFF88014DFF86C04406800F075FADFF8C3
S1133970740400F02CFBDFF8700400F028FBDFF87F
S11339806414DFF850040068000EC0B200F053FA6B
S1133990DFF85814DFF83C040068000CC0B200F0F3
S11339A04AFADFF84C14DFF82C040068000AC0B2AD
S11339B000F041FADFF83C14DFF818040068C0B2E4
S11339C000F039FADFF81C0400F001FB77A000F0E6
S11339D0FEFADFF800044168DFF8F803006800F03D
S11339E029FB00280FD1DFF8DC0300F0F0FA0520F2
S11339F000F0E3FADFF8C803FEF735F9DFF8AC03AB
S1133A0000210170D0E0DFF8C00300F0E0FADFF835
S1133A109C0303210170C7E0DFF8900300780328BA
S1133A2040F0C280DFF898234FF48071DFF8A803D8
S1133A30FEF79AFADFF8781391F83A12C1F3C0113D
S1133A4011F0010101290EDBDFF8AC0300F0BFFA2D
S1133A50022000F0B2FADFF86803FEF704F9D34855
S1133A6000210170A0E000281AD0DFF89023DFF8CD
S1133A706C13DFF8640300F0D9F8040024B214F1E5
S1133A80010F0DD1DFF8780300F0A1FA032000F054
S1133A9094FACB48FEF7E7F8C4480021017083E0AC
S1133AA024B2012C4CDBD74800F091FACD4924B262
S1133AB0200000F0D1F9CB4800F089FAD24800F098
S1133AC086FAC849C448D0F88001000EC0B200F09C
S1133AD0B2F9C649C048D0F88001000CC0B200F069
S1133AE0AAF9C349BC48D0F88001000AC0B200F06A
S1133AF0A2F9C049B848D0F88001C0B200F09BF9DF
S1133B00B84800F064FA29A000F061FABB4A24B274
S1133B102100B148D0F8800100F088FA00280CD1C7
S1133B20A84800F054FA062000F047FAA448FEF72B
S1133B309AF89E480021017036E0A34800F047FA45
S1133B409B48D0F83C029A49D1F84012884201D1EE
S1133B50012000E00020012826DBAC4800F037FA01
S1133B6000F070FA00280CD1964800F030FA0720D3
S1133B7000F023FA9248FEF776F88C480021017091
S1133B8012E0914800F023FAA14800F020FA8C4892
S1133B90FEF769F89F4800F01AFA84480021017082
S1133BA000F0F9F900F058FA10BD00002E2E2E0096
S1133BB010B50400207800F078FA532804D1607816
S1133BC000F077FA002801D103200FE06078312853
S1133BD001D100200AE06078322801D1012005E0FB
S1133BE06078332801D1022000E0032010BD70B5B5
S1133BF004000026A41C200000F047F90500AE19BB
S1133C00A41C200000F041F986196D1EA41CADB25D
S1133C10022DF6DAF6B2F643200000F036F9F6B2D9
S1133C20864201D0002000E0012070BD2DE9F04162
S1133C3005000E0014005FF00008002E01D0002DD6
S1133C4004D140F236215B48FFF764FD2800FFF7FA
S1133C50AFFF0700FFB2032F01D10020A3E028002B
S1133C60FFF7C5FF002802D15FF0FF309BE0FFB2F1
S1133C70002F03D0022F5AD028D392E0AD1C280085
S1133C8000F003F90700AD1C280000F0FEF8000264
S1133C903060AD1CD6F80080280000F0F6F810EB78
S1133CA008003060AD1CB7F10308002C0DD00026CD
S1133CB006E0280000F0E9F8B6B23055AD1C761CD9
S1133CC0B6B20FFA88F84645F3DB6AE0AD1C28006B
S1133CD000F0DBF80700AD1C280000F0D6F8000463
S1133CE03060AD1CD6F80080280000F0CEF818EB48
S1133CF000203060AD1CD6F80080280000F0C5F824
S1133D0010EB08003060AD1CB7F10408002C0DD096
S1133D10002606E0280000F0B8F8B6B23055AD1C15
S1133D20761CB6B20FFA88F84645F3DB39E0AD1CD1
S1133D30280000F0AAF80700AD1C280000F0A5F840
S1133D4000063060AD1CD6F80080280000F09DF815
S1133D5018EB00403060AD1CD6F80080280000F05D
S1133D6094F818EB00203060AD1CD6F800802800D1
S1133D7000F08BF810EB08003060AD1CB7F10508BB
S1133D80002C0DD0002606E0280000F07EF8B6B224
S1133D903055AD1C761CB6B20FFA88F84645F3DBF5
S1133DA0FFE7404600B2BDE8F0810000430F002069
S1133DB004000020EC580000A059000078590000CD
S1133DC038020020505B0000585B0000C45900001A
S1133DD01C590000200F00208C0C00200C0E002029
S1133DE0245B0000E00E0020545A0000E20E002084
S1133DF0E40E0020E60E0020E85900008C0D00209F
S1133E000C5A0000E85A0000A85A0000705A00003A
S1133E10C05A00004C59000080B5010011F00F0099
S1133E203030C9B20A2901DBC01D02E0C0B200F083
S1133E303CF9C0B202BD38B504000D00E4B220095B
S1133E40FFF7EAFF287014F00F00FFF7E5FF687032
S1133E500020A870280032BD0200491C0A23B2FBCE
S1133E60F3F2002AF9D100220A700200491E0A2046
S1133E70B2FBF0F300FB1320303008700A20B2FBD1
S1133E80F0F2002AF2D10800704770B50400002552
S1133E90002609E03038C0B20A2800DBC01FEDB2AA
S1133EA0C0B210EB0515761CF6B2022E0FDAF6B28C
S1133EB0305D00F0FAF8C0B2B0F13001172904D235
S1133EC0C0B2B0F13A010729E4D2002001E0280091
S1133ED0C0B270BD80B515480088ADF8000000F090
S1133EE001F900F02BFB12480078012802D100A848
S1133EF000F022F901BD80B50E4800F057FB0128FF
S1133F0002D10C4800F018F901BD704780B5C9B260
S1133F1000F022FB00F00AF901BD054801210170FF
S1133F207047034800210170704700003A450000C3
S1133F30480F0020A00E002080B500F0EEF802BD6E
S1133F4000B589B000A8202100F092FB00A93148F7
S1133F50FDF772FF002808D10098002805D09DF8CD
S1133F600800C00601D4012000E0002009B000BD13
S1133F702848704780B52848002180F824120A2276
S1133F8026492548FDF744FB002803D12248012196
S1133F9080F8241201BD80B51F4890F8240201283E
S1133FA002D11D48FDF75FFE1D4800F073FC012897
S1133FB0FAD01848FDF76AFF01BD80B5164890F89D
S1133FC02402012802D11448FDF74DFE01BD10B5AD
S1133FD00400114890F82402012817D10E4920004A
S1133FE0FEF705F8002811D50B48002180F82412AB
S1133FF00948FDF738FE09E02178094800F034FC4F
S1134000074800F006FC0028FAD0641C2078002839
S1134010F2D110BD8C5A00005C040020F85A000054
S113402000C0004080B500F063FC01BD80B500F025
S11340306AFC02BD80B500F090FC02BD80B500F0C2
S1134040E9FC02BD80B500F0A2FC002801D10020EB
S113405001E000F007FD02BD80B5FFF7EFFF002887
S11340600BD0FFF752FFFFF738FB04484FF4C04171
S1134070016046F204000068804701BD08ED00E0DD
S113408070B504000D00160005E0287820706D1C42
S1134090641CFFF74CFB3000461E80B20028F4D1AC
S11340A070BD80B500F044FE01BD80B500F04CFE4B
S11340B002BD30380A2801D2012000E00020C0B23D
S11340C0704750F8041B61B150F8042BD30744BF68
S11340D0A9F101039A18002342F8043B091FFAD1FD
S11340E0EFE77047DFF8340400210170DFF82C0497
S11340F000218164DFF82404002180F84310DFF8F4
S11341001C040021A0F84410DFF810040021817081
S1134110DFF80804002141707047DFF800040078DC
S1134120002801D1002000E001207047DFF8EC03F3
S1134130002180F84310704780B50178FF2918D119
S113414000F08BF8DFF8D40390F84300012802D183
S1134150102000F078F8DFF8C403012180F8431040
S1134160DFF8B803B0F94410DFF8B40300F053F8F3
S113417001BDDFF8A813097801294BD10178C929B9
S113418032D0CC293FD0CF293AD0D0292FD0D12931
S113419033D0D2292ED0F32917D0F4290FD0F52902
S11341A00AD0F6290ED0FA2912D0FC2913D0FD2901
S11341B014D0FE2915D029E000F0D5F8C2E700F0AC
S11341C0F1F8BFE700F0C4F8BCE700F00DF9B9E777
S11341D000F0A6F8B6E700F09DF8B3E700F082F827
S11341E0B0E700F070F8ADE700F02FF9AAE700F0AF
S11341F046F9A7E700F00FF9A4E700F06EF9A1E78C
S113420000F07FF99EE700F093F99BE7202000F08F
S11342101AF897E7ACE780B589B2FFF777FE01BDDE
S113422010B4002302E00478E318401C0C00611E63
S1134230002CF8D1DBB21360012010BC7047B748E2
S1134240002141707047B549FE22CA70B349087114
S1134250B2480221A0F84410704710B50400FFF7DB
S11342607AFA002803D11020FFF7EDFF2AE0FFF7C8
S1134270E6FFAA4801210170A848FF21C170A748A0
S113428000210171A548007950F01000A34908717C
S1134290A24800214171A148A049497941719F4830
S11342A0402181719D484021C1719C4800210172C7
S11342B09A48012141729948012181729748082145
S11342C0A0F8441010BD10B50400944800210170FA
S11342D0FFF7B5FF9148FF21C17090480121A0F874
S11342E0441010BD8D49FF22CA708C4900220A7106
S11342F08A498A4A52784A71884900228A718749D0
S11343000022CA71854900220A7284490622A1F852
S11343104420704710B504000020FFF794FF10BD3F
S11343207E49FF22CA707D497E4A8A647B49002205
S11343300A717A4900224A71784900228A717749C0
S11343400722C1F8072075490822A1F844207047C4
S11343507249FF22CA707149406888646F4801211C
S1134360A0F84410704710B504006078402803DBBF
S11343702220FFF768FF14E0627892B26748816CEC
S11343806948FFF77DFE6548FF21C1706348806C72
S113439061780818614988646078401C5F49A1F815
S11343A0440010BD10B504006078402803DB2220CF
S11343B0FFF749FF17E0594861688164627892B257
S11343C05648816C5848FFF75BFE5448FF21C17082
S11343D05248806C61780818504988646078401CA1
S11343E04E49A1F8440010BD80B54C49FF22CA7063
S11343F04E4A41684948806CFFF712FF47490871EB
S113440046480021417145480021817143480821F3
S1134410A0F8441001BD4149FF22CA703F4900225F
S11344200A713E4900224A713C4940228A713B4943
S11344300022CA71394900220A72384900224A729C
S113444036490722A1F84420704780B5421C3F2119
S11344503248806CFFF7EAFD002803D13120FFF7D2
S1134460F2FE0BE02D48FF21C1702C48806C3F30D8
S11344702A49886429480121A0F8441001BD10B5D7
S1134480040060783F2803DB2220FFF7DCFE23E0F2
S11344902248FF21C17021480121A0F8441060780E
S11344A0002807D1FFF7CEFD002802D13120FFF705
S11344B0CAFE11E0A21C61781848806CFFF7B6FDB3
S11344C0002803D13120FFF7BEFE05E01348806CBD
S11344D0617808181149886410BD80B541680F4897
S11344E0806CFFF7A7FD002803D13120FFF7ABFE56
S11344F006E00A48FF21C17008480121A0F84410D1
S113450001BD10B50400FFF7CCFD0448FF21C170C4
S113451002480121A0F8441010BD0000100E002034
S1134520130E0020605B0000140E0020170E002004
S113453080B53120FFF787FE01BDFF0080B54548F7
S1134540FEF70CFEFEF788FF60234FF46142010082
S1134550414800F0B6F801BD70B504000D00EDB29D
S1134560412D03DB56213D48FFF7D4F82800C0B2A3
S113457000F05CF8012803D059213848FFF7CAF845
S113458000260CE0FFF7D3F8B6B2305D00F04EF829
S1134590012803D061213148FFF7BCF8761C2800BC
S11345A0C0B2B6B280B28642ECD370BD10B504007E
S11345B02B48007800280CD12A4800F02AF801285A
S11345C005D12748012101702748002101700020EE
S11345D010BD2548007823494018401C00F019F804
S11345E00128F4D120480078401C1F4908701E4857
S11345F000781C4909788842E9D11B48027892B2B4
S11346001A492000FFF73CFD1548002101700120E4
S1134610DEE710B50400104800F011F910F1010FA5
S113462002D02070012000E0002010BD80B5010000
S1134630C9B2094800F018F9002803D1002007E0A6
S1134640FFF775F8044800F0E4F80028F8D00120DA
S113465002BD00000100001000C00040B05800007E
S1134660450F00205C0E0020440F00205D0E00204A
S1134670002200F075BB0000DFF83C1288421BD01A
S1134680DFF83812884217D0DFF83412884213D08A
S1134690DFF8301288420FD0DFF82C1288420BD09A
S11346A0DFF82812884207D0DFF82412884203D0AA
S11346B0DFF82012884201D1012000E00020C0B2BE
S11346C07047F8B504000E0017001D002000FFF726
S11346D0D3FF002805D14FF4B071DFF8FC01FFF7D8
S11346E019F8002F05D140F26111DFF8EC01FFF752
S11346F011F8DFF8E801006810F0E04F27D0DFF888
S1134700DC010068DFF8D8110840B0F1805F1ED0EA
S1134710DFF8C8010068DFF8C8110840DFF8C411E9
S1134720884205D1DFF8B401006880B202280ED0B7
S1134730DFF8A8010068DFF8A8110840DFF8A81125
S1134740884206D1DFF894010068000401D11020EA
S113475000E0082000FB07F0864205D24FF4B17157
S1134760DFF87401FEF7D6FF200000F038F8B6EB4E
S1134770071F05D2206B50F0200020637F0803E060
S1134780206B30F020002063F000B0FBF7F0401CF9
S11347904008810961624021B0FBF1F202FB110281
S11347A0A262E5620020A061200000F001F8F1BDE2
S11347B010B504002000FFF75FFF002805D14FF477
S11347C0FB71DFF81401FEF7A5FFE06A50F010005A
S11347D0E062206B40F201310843206310BD10B544
S11347E004002000FFF748FF002805D140F21621FD
S11347F0DFF8E400FEF78EFFA0690007FCD4E06A4E
S113480030F01000E062206BDFF8E0100840206315
S113481010BD10B504002000FFF72EFF002805D1BD
S113482040F25541DFF8B000FEF774FFA069C0F311
S1134830401010F0010090F00100C0B210BD10B59E
S113484004002000FFF718FF002805D140F276414C
S1134850DFF88400FEF75EFFA069C00601D420687B
S113486001E05FF0FF3010BD38B504000D002000FA
S1134870FFF702FF002804D140F2C9411648FEF7B1
S113488049FFA069800603D4EDB22560012000E051
S1134890002032BD10B504002000FFF7EDFE002813
S11348A004D140F23B510C48FEF734FFA069C0F339
S11348B0C00010F0010010BD00C0004000D0004056
S11348C000E0004000F00040000001400010014002
S11348D000200140003001405457000000E00F4028
S11348E00000FF700000011000000310FEFCFFFF39
S11348F0DFF830045FF0FF310160DFF82C045FF073
S1134900FF310160704770B504000D0016002000EF
S113491000F0A5F9FF2805D02819401E00F09FF9E2
S1134920FF2801D1002017E0600A4FF400714843CA
S1134930DFF8F8130968884207D12B003200210000
S1134940DFF8E40300F0E1F806E02B003200210078
S1134950DFF8D00300F0D9F870BD70B504000D0085
S1134960200000F07CF906002819401E00F077F9B9
S1134970F6B2FF2E02D0C0B2FF2801D1002005E01C
S11349800100C9B23000C0B200F02CF970BD80B58E
S113499000200090DFF89003006810F1010F01D1AE
S11349A0012036E00098DFF8801349680818009069
S11349B00098DFF874138968081800900098DFF8ED
S11349C06813C968081800900098DFF85C13096937
S11349D0081800900098DFF85013496908180090EF
S11349E00098DFF844138969081800900098DFF8EC
S11349F03813C969081800900098C04300900098C3
S1134A00401C009000AA0421C8480068F030FFF759
S1134A107AFF02BD0020C549096809680818C3491E
S1134A20096849680818C149096889680818BF49AC
S1134A300968C9680818BD49096809690818BB49A3
S1134A40096849690818B949096889690818B7499A
S1134A500968D1F8F0100818002801D1012000E0FD
S1134A600020704780B5B048006810F1010F06D0EF
S1134A70AD4800F08DF8002801D100200CE0A948D1
S1134A80006810F1010F06D0A64800F081F8002854
S1134A9001D1002000E0012002BD80B54FF4007276
S1134AA0B1FBF2F303FB1213002B01D000200BE047
S1134AB002688A4201D1012006E001604FF40072CD
S1134AC0001DFFF7DDFA012002BD38B504000D001A
S1134AD09548844208D1934C29002000FFF7DDFF5C
S1134AE0002810D100200FE090480068854203D1CF
S1134AF08D4C8E480568EFE7200000F049F8002847
S1134B00EAD1002000E0200032BD2DE9F04104008C
S1134B100F0015001E00780A4FF4007101FB00F825
S1134B20206810F1010F07D141462000FFF7B5FFBF
S1134B30002801D1002029E02068404508D04146E2
S1134B402000FFF7C2FF0400002C01D100201DE06B
S1134B502068381A0019071DFEF7E9FD201D381AD0
S1134B60B0F5007F0AD318F500712000FFF7ADFF00
S1134B700400002C01D1002008E0271D287838709B
S1134B807F1C6D1C761E002EE6D10120BDE8F0814D
S1134B90F8B505000124286800F061F8C0B2FF28C8
S1134BA001D100201DE0002600E0761C802E16D2E4
S1134BB0286810EB860715EB860040680090FEF726
S1134BC0B6FD0422390000A800F00BF9002801D03A
S1134BD0002404E0386800998842E6D000242000CC
S1134BE0C0B2F2BD70B50D00EDB2C0B2854201D2C3
S1134BF0002033E04D49097AC0B2884205D34B49BD
S1134C0091F8C810EDB2A94201D2002026E0C0B24A
S1134C1000F04FF804002800C0B200F04AF8060083
S1134C202800C0B200F062F88019401E001B401C2E
S1134C30850A002600E0761CB6B2ADB2AE420CD2B4
S1134C40FEF775FDB6B24FF4806000FB064000F03D
S1134C50A1F80028EFD0002000E0012070BD38B595
S1134C600400002500E06D1CEDB2112D1FD2FEF7EB
S1134C705EFDEDB20C202D4900FB05100068844256
S1134C80F1D3EDB20C20294900FB05100068EDB208
S1134C900C21264A01FB0521496808188442E2D206
S1134CA0EDB20C20214900FB0510007A00E0FF2042
S1134CB032BD38B50400002500E06D1CEDB2112DA5
S1134CC011D2FEF734FDEDB20C20184900FB05109B
S1134CD0007AE4B2A042F0D1EDB20C20134900FBFB
S1134CE00510006801E05FF0FF3032BD38B5040004
S1134CF0002500E06D1CEDB2112D11D2FEF717FD59
S1134D00EDB20C20094900FB0510007AE4B2A04280
S1134D10F0D1EDB20C20054900FB0510406800E01D
S1134D20002032BD8406002088080020DC540000E6
S1134D30044B9D46C046C046C046C046FFF7F1F846
S1134D4000F0CEF85011002010B50400200000F04F
S1134D50D2F8002801D0203CFFE7200010BD00005D
S1134D6000B500BF130096469446103928BFA0E84A
S1134D700C50FAD85FEA417C28BF0CC048BF40F809
S1134D80042BC90728BF20F8022B48BF00F8012BC9
S1134D9000BD000010B50400A00504D09C21DFF87C
S1134DA01001FEF7B7FCDFF80C0140F601210160A9
S1134DB0DFF804010460DFF80401DFF80411016086
S1134DC0DFF8F80000688007FAD4DFF8F80000681C
S1134DD040F60121084202D05FF0FF3000E00020DD
S1134DE010BD70B504000D00160015F0030F04D0BB
S1134DF0DF21DFF8BC00FEF78DFC16F0030F04D0B2
S1134E00E021DFF8AC00FEF785FCDFF8A80042F2F1
S1134E1001610160DFF8B0000068C00739D5002ED9
S1134E2039D0E809C001DFF89010086008E015F0F7
S1134E307C00DFF8981022680A50241D2D1D361FAF
S1134E4015F07C0F04D1DFF888000068002801D138
S1134E50002EECD1DFF87C00DFF87C100160DFF875
S1134E6074000068C007FAD4D9E7DFF84C00056085
S1134E70DFF8680021680160DFF84000DFF85810AF
S1134E800160DFF838000068C007FAD4241D2D1D26
S1134E90361F002EE9D1DFF82C00006842F20161D0
S1134EA0084202D05FF0FF3000E0002070BD000037
S1134EB09456000014D00F4000D00F4008D00F408B
S1134EC0020042A40CD00F40A0E10F4000D10F40DB
S1134ED030D00F4020D00F40010042A404D00F4036
S1134EE000F011F8002801D000F010F8002000F0C4
S1134EF021F800F039F861381A2801D2012000E0C5
S1134F000020C0B2704701207047000010B5074967
S1134F1079441831064C7C44163404E00A68081DB0
S1134F20511888470146A142F8D110BD040B000076
S1134F30240B000080B500F005F800F017F800F02D
S1134F4023F8FCE780B50648FEF782F90548FEF72A
S1134F5005F903215FF04020FDF794FE01BD000038
S1134F608003C0010100002000F01AB880B5FEF7EC
S1134F70DDFBFEF7A1FBFFF755F8FEF7D9FBFEF7C3
S1134F80A9FF00F013F801BD80B5FEF7D0FBFEF7D2
S1134F90A8FBFEF703FCFEF7AEFF00F012F801BD1C
S1134FA00746384600F030F8FBE7000080B51448A7
S1134FB001210170FEF79FFB1249086000F001F81F
S1134FC001BD80B5FEF7B8FF012817D0FEF7C3FB7B
S1134FD0002813D00A48007801280FD1FEF78BFB74
S1134FE0084909683231884208D305480021017014
S1134FF0FEF7BAFB002801D1FFF72EF801BD00002F
S1135000420F0020300F002080B5C046C046024A3F
S113501011001820ABBEFBE726000200610062000D
S113502063006400650066006700680069006A0048
S11350306B006C006D006E006F00700071007200F8
S113504073007400750076007700780079007A00A8
S1135050A100A200A300A500AC00AF00E000E100A5
S1135060E200E300E400E500E600E700E800E90010
S1135070EA00EB00EC00ED00EE00EF00F000F100C0
S1135080F200F300F400F500F600F800F900FA006D
S1135090FB00FC00FD00FE00FF000101030105010F
S11350A0070109010B010D010F0111011301150184
S11350B0170119011B011D011F01210123012501F4
S11350C0270129012B012D012F0131013301350164
S11350D037013A013C013E014001420144014601CD
S11350E048014B014D014F01510153015501570135
S11350F059015B015D015F016101630165016701A4
S113510069016B016D016F01710173017501770113
S11351107A017C017E019201B103B203B303B403AB
S1135120B503B603B703B803B903BA03BB03BC039F
S1135130BD03BE03BF03C003C103C303C403C5034C
S1135140C603C703C803C903CA03300431043204C5
S113515033043404350436043704380439043A0477
S11351603B043C043D043E043F0440044104420427
S113517043044404450446044704480449044A04D7
S11351804B044C044D044E044F0451045204530484
S11351905404550456045704580459045A045B042F
S11351A05C045E045F0470217121722173217421F7
S11351B0752176217721782179217A217B217C211F
S11351C07D217E217F2141FF42FF43FF44FF45FFB4
S11351D046FF47FF48FF49FF4AFF4BFF4CFF4DFF87
S11351E04EFF4FFF50FF51FF52FF53FF54FF55FF37
S11351F056FF57FF58FF59FF5AFF00004100420075
S113520043004400450046004700480049004A0066
S11352104B004C004D004E004F0050005100520016
S113522053005400550056005700580059005A00C6
S11352302100E0FFE1FFE5FFE2FFE3FFC000C10062
S1135240C200C300C400C500C600C700C800C9002E
S1135250CA00CB00CC00CD00CE00CF00D000D100DE
S1135260D200D300D400D500D600D800D900DA008B
S1135270DB00DC00DD00DE00780100010201040136
S1135280060108010A010C010E01100112011401AA
S1135290160118011A011C011E012001220124011A
S11352A0260128012A012C012E013001320134018A
S11352B0360139013B013D013F01410143014501F3
S11352C047014A014C014E0150015201540156015B
S11352D058015A015C015E016001620164016601CA
S11352E068016A016C016E0170017201740176013A
S11352F079017B017D01910191039203930394034E
S1135300950396039703980399039A039B039C03BD
S11353109D039E039F03A003A103A303A403A5036A
S1135320A603A703A803A903AA03100411041204E3
S113533013041404150416041704180419041A0495
S11353401B041C041D041E041F0420042104220445
S113535023042404250426042704280429042A04F5
S11353602B042C042D042E042F0401040204030432
S11353700404050406040704080409040A040B04CD
S11353800C040E040F046021612162216321642155
S1135390652166216721682169216A216B216C21BD
S11353A06D216E216F2121FF22FF23FF24FF25FFA2
S11353B026FF27FF28FF29FF2AFF2BFF2CFF2DFFA5
S11353C02EFF2FFF30FF31FF32FF33FF34FF35FF55
S11353D036FF37FF38FF39FF3AFF0000C700FC00F3
S11353E0E900E200E400E000E500E700EA00EB0089
S11353F0E800EF00EE00EC00C400C500C900E600C0
S1135400C600F400F600F200FB00F900FF00D6002D
S1135410DC00A200A300A500A7209201E100ED009A
S1135420F300FA00F100D100AA00BA00BF00102373
S1135430AC00BD00BC00A100AB00BB0091259225CF
S113544093250225242561256225562555256325A6
S1135450512557255D255C255B251025142534250C
S11354602C251C2500253C255E255F255A25542521
S113547069256625602550256C25672568256425E2
S1135480652559255825522553256B256A25182548
S11354900C25882584258C2590258025B103DF00E3
S11354A09303C003A303C303B500C403A603980373
S11354B0A903B4031E22C603B50329226122B10045
S11354C06522642220232123F7004822B0001922F8
S11354D0B7001A227F20B200A025A00000600000BF
S11354E000200000030000000080000000200000F5
S11354F00400000000A000000020000005000000DF
S113550000C00000002000000600000000E00000D1
S1135510002000000700000000000100002000003F
S11355200800000000200100002000000900000025
S113553000400100002000000A000000006001009B
S1135540002000000B00000000800100002000008B
S11355500C00000000A00100002000000D0000006D
S113556000C00100002000000E00000000E0010067
S1135570002000000F000000000002000080000076
S113558010000000008002000080000011000000F4
S113559000000300008000001200000000800300EF
S11355A00080000013000000809A90418E418F809B
S11355B04545454949498E8F9092924F994F55558B
S11355C059999A9B9C9D9E9F41494F55A5A5A6A775
S11355D0A8A9AAABAC21AEAFB0B1B2B3B4B5B6B75B
S11355E0B8B9BABBBCBDBEBFC0C1C2C3C4C5C6C7BF
S11355F0C8C9CACBCCCDCECFD0D1D2D3D4D5D6D7AF
S1135600D8D9DADBDCDDDEDFE0E1E2E3E4E5E6E79E
S1135610E8E9EAEBECEDEEEFF0F1F2F3F4F5F6F78E
S1135620F8F9FAFBFCFDFEFF40420F0000201C00CD
S113563080841E0000802500999E360000403800BA
S113564000093D0000803E0000004B00404B4C0030
S113565000204E00808D5B0000C05D000080700063
S113566000127A0000007D0080969800001BB700AD
S11356700080BB00C0E8CE00647ADA000024F400A5
S11356800000FA0080A81201002D310100366E01DD
S113569040787D01433A5C576F726B5C736F66743C
S11356A0776172655C4F70656E424C545C546172F4
S11356B06765745C44656D6F5C41524D434D335F67
S11356C04C4D33535F454B5F4C4D33533639363570
S11356D05F4941525C426F6F745C6C69625C6472D6
S11356E0697665726C69625C666C6173686C696228
S11356F02E630000433A5C576F726B5C736F667481
S1135700776172655C4F70656E424C545C54617293
S11357106765745C44656D6F5C41524D434D335F06
S11357204C4D33535F454B5F4C4D3353363936350F
S11357305F4941525C426F6F745C6C69625C647275
S1135740697665726C69625C73797363746C2E63D9
S113575000000000433A5C576F726B5C736F6674B1
S1135760776172655C4F70656E424C545C54617233
S11357706765745C44656D6F5C41524D434D335FA6
S11357804C4D33535F454B5F4C4D335336393635AF
S11357905F4941525C426F6F745C6C69625C647215
S11357A0697665726C69625C756172746C69622E8B
S11357B063000000433A5C576F726B5C736F6674EE
S11357C0776172655C4F70656E424C545C546172D3
S11357D06765745C44656D6F5C41524D434D335F46
S11357E04C4D33535F454B5F4C4D3353363936354F
S11357F05F4941525C426F6F745C6C69625C6472B5
S1135800697665726C69625C6770696F2E6300000B
S1135810433A5C576F726B5C736F66747761726541
S11358205C4F70656E424C545C5461726765745C85
S113583044656D6F5C41524D434D335F4C4D335362
S11358405F454B5F4C4D3353363936355F494152D2
S11358505C426F6F745C6C69625C647269766572D9
S11358606C69625C7373692E63000000433A5C5791
S11358706F726B5C736F6674776172655C4F706591
S11358806E424C545C5461726765745C536F7572FC
S113589063655C41524D434D335F4C4D33535C491A
S11358A041525C766563746F72732E63000000006E
S11358B0433A5C576F726B5C736F667477617265A1
S11358C05C4F70656E424C545C5461726765745CE5
S11358D0536F757263655C41524D434D335F4C4D5C
S11358E033535C756172742E63000000433A5C5755
S11358F06F726B5C736F6674776172655C4F706511
S11359006E424C545C5461726765745C536F75727B
S113591063655C66696C652E630000005061727398
S1135920696E67206669726D776172652066696C5D
S11359306520746F206F627461696E206572617393
S1135940652073697A652E2E2E0000004669726DFB
S11359507761726520757064617465207375636323
S113596065737366756C6C7920636F6D706C6574A8
S113597065640A0D000000004F70656E696E672053
S11359806669726D776172652066696C6520666F01
S1135990722072656164696E672E2E2E000000000D
S11359A04669726D776172652075706461746520F3
S11359B07265717565737420646574656374656478
S11359C00A0D00005374617274696E67207468650F
S11359D02070726F6772616D6D696E672073657197
S11359E075656E63650A0D0052656164696E6720B2
S11359F06C696E652066726F6D2066696C652E2E0B
S1135A002E4552524F520A0D00000000496E766135
S1135A106C696420636865636B73756D20666F756C
S1135A206E642E2E2E4552524F520A0D0000000075
S1135A3093E6FFFF440F0000040000200000000074
S1135A40DBC5FFFF0400000020010000000000206F
S1135A50000000002062797465732066726F6D2007
S1135A606D656D6F727920617420307800000000DC
S1135A7057726974696E672070726F6772616D2006
S1135A80636865636B73756D2E2E2E002F64656DD0
S1135A906F70726F675F656B5F6C6D337336393629
S1135AA0352E737265630000206279746573207407
S1135AB06F206D656D6F72792061742030780000FD
S1135AC0436C6F73696E67206669726D7761726586
S1135AD02066696C650A0D0001030507090E1012A2
S1135AE01416181C1E00000050726F6772616D6DF1
S1135AF0696E6720000000002F626F6F746C6F671F
S1135B002E7478740000000080B541210148FDF72F
S1135B1001FE01BD6C580000222A3A3C3E3F7C7FC6
S1135B200000000045726173696E67200000000088
S1135B3000E10F4004E10F4008E10F40C046C046B9
S1135B40C046C046FFF7CCF92B2C3B3D5B5D000003
S1135B504552524F520A0D004F4B0A0D00000000EF
S10F5B604F70656E424C540001000000C0
S9035B3D64
